:020000040000FA
:02000000462890
:040002000034003492
:08000800A000030EA1008B18FB
:1000100014280B1D41280B11A60A2608063A031DB9
:100020004128A501A60141288B10A50A25080B3AF5
:10003000031D3128A5012214A6012308F03A031953
:10004000222824288403412823088000840A0408E5
:10005000503A03192D28851141284F308400851509
:10006000412825080A3A031941282508013A0319AD
:100070004128A3138618A317A30C2508093A0319CE
:10008000A30D210E8300A00E200E0900E120F9200F
:100090000F30B4002721403084005030B1004C3084
:1000A000C0004C30C1004C30C2005A30C300443054
:1000B00084000B118B108B170408403A03195C283D
:1000C00040080319BA2840085B3A031D6E28063021
:1000D000A7003330A800B1201921BA284008293AD6
:1000E000031D7A280C210C210C210C210C210C2140
:1000F0000C21BA284008073A031D7F2867294008C9
:10010000053A031D8F283108783A03198F283108E2
:10011000053EB100B403192119212721BA2840084E
:10012000063A031D9F2831081E3A03199F283108FB
:10013000FB3EB100B40A192119212721BA28043045
:100140008A000030400703188A0A40080024A700EC
:10015000A800A7080319BA28A70E0F30A705031097
:10016000A70C0310A80C031C07290229A70BB12810
:100170000C210C214108C0004208C1004308C20004
:100180004408C3004508C4004608C5004708C60027
:100190004808C7004908C8004A08C9004B08CA00F7
:1001A0004C08CB004D08CC004E08CD004F08CE00C7
:1001B0000408403A031DDF28DD28C0015C288403C1
:1001C0005C2800308500860007309F00831684304D
:1001D0008100003085000330860000308C00003044
:1001E0009F00831230308B0000308C000030900074
:1001F0000800203084008001840A0408603A031D4E
:10020000FB28080086150C2186110C21B6288615BE
:10021000192186110C21B6283108B0004B30A900F5
:100220000230AA00A90B1229AA0B1229B00B0E2921
:1002300008003108B000E430A9000430AA00A90B7E
:100240001F29AA0B1F290000B00B1B29080005104D
:100250000830AF00B2013408B20AF63E03182C2968
:10026000B2030A3EB30001308A005A303207031845
:100270008A0A32085A21B20001308A005A30330704
:1002800003188A0A33085A21B3008510B31B85145A
:10029000B30D05140510AF0B45290830AF008510CC
:1002A000B21B8514B20D05140510AF0B4F290515AF
:1002B00005110800000082073F3406345B344F34D8
:1002C00066346D347D3407347F346F340800BA28C7
:1008000082070034003400340034003400340034F3
:100810000034003400340034003400340034003438
:100820000034003400340034003400348134A13406
:10083000003400340034853482348B348A34A33459
:10084000003400346734883461346334AF34A734FF
:100850000034003400344034413421346234BF3435
:100860000034003420344334653489344234BE3497
:10087000003400340034863460346434BC34B8341A
:10088000003400348E348D3480348434A034B03459
:100890000034003483340034663487348C340034BC
:1008A000003400340034BB3400348F34003400345E
:1008B000003400340034AE34863400340034003464
:1008C0000034003400340034003400340034003488
:1008D0000034003400340034003400340034003478
:1008E0000034003400340034003400340034003468
:1008F0000034003400340034003400340034003458
:100900000034003400340034003400340034003447
:100910000034003400340034003400340034003437
:100920000034003400340034003400340034003427
:100930000034003400340034003400340034003417
:100940000034003400340034003400340034003407
:1009500000340034003400340034003400340034F7
:1009600000340034003400340034003400340034E7
:1009700000340034003400340034003400340034D7
:1009800000340034003400340034003400340034C7
:1009900000340034003400340034003400340034B7
:1009A00000340034003400340034003400340034A7
:1009B0000034003400340034003400340034003497
:1009C0000034003400340034003400340034003487
:1009D0000034003400340034003400340034003477
:1009E0000034003400340034003400340034003467
:1009F0000034003400340034003400340034003457
:0E0A000000340034003400340034003400347C
:02400E00303F41
:00000001FF
